:10000000250003023200A30404006100DF0C02009B
:100010000400DC0C020004006600C90C0600920714
:100020008605A305000B28050606AB020806970AFD
:10003000AC024306EC000606AB020000A709060668
:10004000AB020A0243074605430646040606AB0216
:1000500029000606130A2806330A6B000606AB02BF
:100060000806970A1B0A0B022F00030C8C000307DB
:10007000E8050307EF06E804A709000000000A02EC
:1000800043074605430646042900080C8C00030676
:10009000E8056C00800CAF00BA0C8F000306E80581
:1000A000E806880A1002EF012F03A70900000000EC
:1000B0000A02430746054306460429000F02A50924
:1000C000A3042D003F0E2A00CD06720A260400006C
:1000D000A709190C31000A024307460543064604E6
:1000E0002900780A4604A709F102780AB102260518
:1000F0000F023000040000000000000000000000BB
:10010000000000000000000028046B00A709210A7D
:10011000A6050000A709A604E8040A02430746054D
:100120004306460429000000000000007B0A460444
:10013000190C3100040006079A0A040006069D0AFD
:10014000F1029A0A2605A305000BA3052200660703
:1001500008050606AB02E9004306460466070805E3
:100160000606AB02E90043064604660708050606D4
:10017000AB02E90043064604660708050606AB0223
:10018000E90043064604660708050606AB02E900D7
:1001900043064604660708050606AB02E900430667
:1001A0004604660708050606AB02E9004306460456
:1001B000660708050606AB02E90043064604660723
:1001C00008050606AB02E900430646046607080573
:1001D0000606AB02E9004306460466070805060664
:1001E000AB02E90043064604660708050606AB02B3
:1001F000E90043064604660708050606AB02E90067
:1002000043064604660708050606AB02E9004306F6
:100210004604660708050606AB02E90043064604E5
:10022000660708050606AB02E900430646046607B2
:1002300008050606AB02E900430646046607080502
:100240000606AB02E90043064604660708050606F3
:10025000AB02E90043064604660708050606AB0242
:10026000E90043064604660708050606AB02E900F6
:1002700043064604660708050606AB02E900430686
:100280004604660708050606AB02E9004306460475
:10029000660708050606AB02E90043064604660742
:1002A00008050606AB02E900430646046607080592
:1002B0000606AB02E9004306460466070805060683
:1002C000AB02E90043064604660708050606AB02D2
:1002D000E90043064604660708050606AB02E90086
:1002E00043064604660708050606AB02E900430616
:1002F0004604660708050606AB02E9004306460405
:10030000660708050606AB02E900430646046607D1
:1003100008050606AB02E900430646046607080521
:100320000606AB02E9004306460466070805060612
:10033000AB02E90043064604660708050606AB0261
:10034000E90043064604660708050606AB02E90015
:1003500043064604660708050606AB02E9004306A5
:100360004604660708050606AB02E9004306460494
:10037000660708050606AB02E90043064604660761
:1003800008050606AB02E9004306460466070805B1
:100390000606AB02E90043064604660708050606A2
:0A03A000AB02E90043064604000822
:1004000040084008400840084008400840084008AC
:10041000400840084008400840084008400840089C
:10042000400840084008400840084008400840088C
:10043000400840084008400840084008400840087C
:10044000400840084008400840084008400840086C
:100450004008400840080008000800080308050894
:100460000608070809080A080A080B080C080D08FE
:100470000E080E080F0810081008110812081208BC
:100480001308130814081508150816081608170885
:100490001708180818081908190819081A081A0856
:1004A0001B081B081C081C081C081D081D081E082A
:1004B0001E081E081F081F08200820082008210801
:1004C00021082108220822082208230823082308DB
:1004D00024082408240825082508250826082608B5
:1004E0002608270827082708280828082808280891
:1004F0002908290829082A082A082A082B082B086D
:100500002B083F083F083F083F083F083F083F08C7
:100510003F083F083F083F083F083F083F083F08A3
:100520003F083F083F083F083F083F083F083F0893
:100530003F083F083F083F083F083F083F083F0883
:100540003F083F083F083F083F083F083F083F0873
:100550003F083F083F083F083F083F083F083F0863
:100560003F083F083F083F083F083F083F083F0853
:100570003F083F083F083F083F083F083F083F0843
:100580003F083F083F083F083F083F083F083F0833
:100590003F083F083F083F083F083F083F083F0823
:1005A0003F083F083F083F083F083F083F083F0813
:1005B0003F083F083F083F083F083F083F083F0803
:1005C0003F083F083F083F083F083F083F083F08F3
:1005D0003F083F083F083F083F083F083F083F08E3
:1005E0003F083F083F083F083F083F083F083F08D3
:1005F0003F083F083F083F083F083F083F083F08C3
:1006000004006607000B6607000B0607030B66076E
:10061000000B0606070B050C2E006B000400660796
:10062000000B06070F0BAB024306000B000006068B
:10063000130B0400800CAB002B0C8B000306030B88
:10064000EE020D0B260469004605000000000000C4
:10065000000000000000000000000000000000009A
:1006600000000000A60500000000000000000000DF
:10067000000000000000000000000000000000007A
:1006800046043C0C2A000400EA02430BA6043C0C7E
:100690002A000400EA02490BE902240B06074E0B6C
:1006A0000606500B6A006B006C0070006800190CA5
:0606B0003100A3041B0A47
:021FFE00EE0FE4
:00000001FF
